Archive member included because of file (symbol)

e:/winavr-20071221/bin/../lib/gcc/avr/4.2.2/avr5\libgcc.a(_divmodhi4.o)
                              ks0108.o (__divmodhi4)
e:/winavr-20071221/bin/../lib/gcc/avr/4.2.2/avr5\libgcc.a(_exit.o)
                              e:/winavr-20071221/bin/../lib/gcc/avr/4.2.2/../../../../avr/lib/avr5/crtm16.o (exit)
e:/winavr-20071221/bin/../lib/gcc/avr/4.2.2/avr5\libgcc.a(_copy_data.o)
                              komparator.o (__do_copy_data)
e:/winavr-20071221/bin/../lib/gcc/avr/4.2.2/avr5\libgcc.a(_clear_bss.o)
                              komparator.o (__do_clear_bss)
e:/winavr-20071221/bin/../lib/gcc/avr/4.2.2/avr5\libgcc.a(_fixunssfsi.o)
                              touch.o (__fixunssfsi)
e:/winavr-20071221/bin/../lib/gcc/avr/4.2.2/avr5\libgcc.a(_addsub_sf.o)
                              e:/winavr-20071221/bin/../lib/gcc/avr/4.2.2/avr5\libgcc.a(_fixunssfsi.o) (__subsf3)
e:/winavr-20071221/bin/../lib/gcc/avr/4.2.2/avr5\libgcc.a(_mul_sf.o)
                              touch.o (__mulsf3)
e:/winavr-20071221/bin/../lib/gcc/avr/4.2.2/avr5\libgcc.a(_gt_sf.o)
                              touch.o (__gtsf2)
e:/winavr-20071221/bin/../lib/gcc/avr/4.2.2/avr5\libgcc.a(_ge_sf.o)
                              e:/winavr-20071221/bin/../lib/gcc/avr/4.2.2/avr5\libgcc.a(_fixunssfsi.o) (__gesf2)
e:/winavr-20071221/bin/../lib/gcc/avr/4.2.2/avr5\libgcc.a(_lt_sf.o)
                              touch.o (__ltsf2)
e:/winavr-20071221/bin/../lib/gcc/avr/4.2.2/avr5\libgcc.a(_sf_to_si.o)
                              e:/winavr-20071221/bin/../lib/gcc/avr/4.2.2/avr5\libgcc.a(_fixunssfsi.o) (__fixsfsi)
e:/winavr-20071221/bin/../lib/gcc/avr/4.2.2/avr5\libgcc.a(_thenan_sf.o)
                              e:/winavr-20071221/bin/../lib/gcc/avr/4.2.2/avr5\libgcc.a(_addsub_sf.o) (__thenan_sf)
e:/winavr-20071221/bin/../lib/gcc/avr/4.2.2/avr5\libgcc.a(_udivmodhi4.o)
                              e:/winavr-20071221/bin/../lib/gcc/avr/4.2.2/avr5\libgcc.a(_divmodhi4.o) (__udivmodhi4)
e:/winavr-20071221/bin/../lib/gcc/avr/4.2.2/avr5\libgcc.a(_prologue.o)
                              e:/winavr-20071221/bin/../lib/gcc/avr/4.2.2/avr5\libgcc.a(_addsub_sf.o) (__prologue_saves__)
e:/winavr-20071221/bin/../lib/gcc/avr/4.2.2/avr5\libgcc.a(_epilogue.o)
                              e:/winavr-20071221/bin/../lib/gcc/avr/4.2.2/avr5\libgcc.a(_addsub_sf.o) (__epilogue_restores__)
e:/winavr-20071221/bin/../lib/gcc/avr/4.2.2/avr5\libgcc.a(_pack_sf.o)
                              e:/winavr-20071221/bin/../lib/gcc/avr/4.2.2/avr5\libgcc.a(_addsub_sf.o) (__pack_f)
e:/winavr-20071221/bin/../lib/gcc/avr/4.2.2/avr5\libgcc.a(_unpack_sf.o)
                              e:/winavr-20071221/bin/../lib/gcc/avr/4.2.2/avr5\libgcc.a(_addsub_sf.o) (__unpack_f)
e:/winavr-20071221/bin/../lib/gcc/avr/4.2.2/avr5\libgcc.a(_fpcmp_parts_sf.o)
                              e:/winavr-20071221/bin/../lib/gcc/avr/4.2.2/avr5\libgcc.a(_gt_sf.o) (__fpcmp_parts_f)
e:/winavr-20071221/bin/../lib/gcc/avr/4.2.2/../../../../avr/lib/avr5\libc.a(itoa.o)
                              komparator.o (itoa)
e:/winavr-20071221/bin/../lib/gcc/avr/4.2.2/../../../../avr/lib/avr5\libc.a(strrev.o)
                              e:/winavr-20071221/bin/../lib/gcc/avr/4.2.2/../../../../avr/lib/avr5\libc.a(itoa.o) (strrev)

Allocating common symbols
Common symbol       size              file

ks0108FontColor     0x1               ks0108.o
ks0108Coord         0x3               ks0108.o
ks0108FontRead      0x2               ks0108.o
ks0108Font          0x2               ks0108.o

Memory Configuration

Name             Origin             Length             Attributes
text             0x00000000         0x00020000         xr
data             0x00800060         0x0000ffa0         rw !x
eeprom           0x00810000         0x00010000         rw !x
fuse             0x00820000         0x00000400         rw !x
lock             0x00830000         0x00000400         rw !x
signature        0x00840000         0x00000400         rw !x
*default*        0x00000000         0xffffffff

Linker script and memory map

LOAD e:/winavr-20071221/bin/../lib/gcc/avr/4.2.2/../../../../avr/lib/avr5/crtm16.o
LOAD komparator.o
LOAD ks0108.o
LOAD touch.o
LOAD e:/winavr-20071221/bin/../lib/gcc/avr/4.2.2/avr5\libgcc.a
LOAD e:/winavr-20071221/bin/../lib/gcc/avr/4.2.2/../../../../avr/lib/avr5\libc.a
LOAD e:/winavr-20071221/bin/../lib/gcc/avr/4.2.2/avr5\libgcc.a

.hash
 *(.hash)

.dynsym
 *(.dynsym)

.dynstr
 *(.dynstr)

.gnu.version
 *(.gnu.version)

.gnu.version_d
 *(.gnu.version_d)

.gnu.version_r
 *(.gnu.version_r)

.rel.init
 *(.rel.init)

.rela.init
 *(.rela.init)

.rel.text
 *(.rel.text)
 *(.rel.text.*)
 *(.rel.gnu.linkonce.t*)

.rela.text
 *(.rela.text)
 *(.rela.text.*)
 *(.rela.gnu.linkonce.t*)

.rel.fini
 *(.rel.fini)

.rela.fini
 *(.rela.fini)

.rel.rodata
 *(.rel.rodata)
 *(.rel.rodata.*)
 *(.rel.gnu.linkonce.r*)

.rela.rodata
 *(.rela.rodata)
 *(.rela.rodata.*)
 *(.rela.gnu.linkonce.r*)

.rel.data
 *(.rel.data)
 *(.rel.data.*)
 *(.rel.gnu.linkonce.d*)

.rela.data
 *(.rela.data)
 *(.rela.data.*)
 *(.rela.gnu.linkonce.d*)

.rel.ctors
 *(.rel.ctors)

.rela.ctors
 *(.rela.ctors)

.rel.dtors
 *(.rel.dtors)

.rela.dtors
 *(.rela.dtors)

.rel.got
 *(.rel.got)

.rela.got
 *(.rela.got)

.rel.bss
 *(.rel.bss)

.rela.bss
 *(.rela.bss)

.rel.plt
 *(.rel.plt)

.rela.plt
 *(.rela.plt)

.text           0x00000000     0x2e76
 *(.vectors)
 .vectors       0x00000000       0x54 e:/winavr-20071221/bin/../lib/gcc/avr/4.2.2/../../../../avr/lib/avr5/crtm16.o
                0x00000000                __vectors
                0x00000000                __vector_default
 *(.vectors)
 *(.progmem.gcc*)
 *(.progmem*)
 .progmem.data  0x00000054      0x534 komparator.o
                0x00000588                . = ALIGN (0x2)
                0x00000588                __trampolines_start = .
 *(.trampolines)
 .trampolines   0x00000588        0x0 linker stubs
 *(.trampolines*)
                0x00000588                __trampolines_end = .
 *(.jumptables)
 *(.jumptables*)
 *(.lowtext)
 *(.lowtext*)
                0x00000588                __ctors_start = .
 *(.ctors)
                0x00000588                __ctors_end = .
                0x00000588                __dtors_start = .
 *(.dtors)
                0x00000588                __dtors_end = .
 SORT(*)(.ctors)
 SORT(*)(.dtors)
 *(.init0)
 .init0         0x00000588        0x0 e:/winavr-20071221/bin/../lib/gcc/avr/4.2.2/../../../../avr/lib/avr5/crtm16.o
                0x00000588                __init
 *(.init0)
 *(.init1)
 *(.init1)
 *(.init2)
 .init2         0x00000588        0xc e:/winavr-20071221/bin/../lib/gcc/avr/4.2.2/../../../../avr/lib/avr5/crtm16.o
 *(.init2)
 *(.init3)
 *(.init3)
 *(.init4)
 .init4         0x00000594       0x16 e:/winavr-20071221/bin/../lib/gcc/avr/4.2.2/avr5\libgcc.a(_copy_data.o)
                0x00000594                __do_copy_data
 .init4         0x000005aa       0x10 e:/winavr-20071221/bin/../lib/gcc/avr/4.2.2/avr5\libgcc.a(_clear_bss.o)
                0x000005aa                __do_clear_bss
 *(.init4)
 *(.init5)
 *(.init5)
 *(.init6)
 *(.init6)
 *(.init7)
 *(.init7)
 *(.init8)
 *(.init8)
 *(.init9)
 .init9         0x000005ba        0x8 e:/winavr-20071221/bin/../lib/gcc/avr/4.2.2/../../../../avr/lib/avr5/crtm16.o
 *(.init9)
 *(.text)
 .text          0x000005c2        0x4 e:/winavr-20071221/bin/../lib/gcc/avr/4.2.2/../../../../avr/lib/avr5/crtm16.o
                0x000005c2                __vector_1
                0x000005c2                __vector_12
                0x000005c2                __bad_interrupt
                0x000005c2                __vector_6
                0x000005c2                __vector_3
                0x000005c2                __vector_11
                0x000005c2                __vector_13
                0x000005c2                __vector_17
                0x000005c2                __vector_19
                0x000005c2                __vector_7
                0x000005c2                __vector_4
                0x000005c2                __vector_9
                0x000005c2                __vector_2
                0x000005c2                __vector_15
                0x000005c2                __vector_8
                0x000005c2                __vector_14
                0x000005c2                __vector_10
                0x000005c2                __vector_18
                0x000005c2                __vector_20
 .text          0x000005c6      0x182 komparator.o
                0x0000071a                __vector_5
                0x000005f0                main
                0x000005c6                __vector_16
 .text          0x00000748     0x162a ks0108.o
                0x00001874                ks0108GotoXY
                0x000015aa                ks0108Puts
                0x000011be                ks0108SetInverted
                0x000019d2                ks0108DoReadData
                0x00001296                ks0108ReadFontData
                0x00000b50                ks0108DrawRect
                0x00001bac                ks0108WriteData
                0x000017fa                ks0108StringWidth_P
                0x00000e5c                ks0108FillRect
                0x00001324                ks0108PutChar
                0x0000100c                ks0108InvertRect
                0x000018fe                ks0108Init
                0x00000bc6                ks0108DrawRoundRect
                0x000016e4                ks0108CharWidth
                0x00001b06                ks0108WriteCommand
                0x00001ae8                ks0108ReadData
                0x00001796                ks0108StringWidth
                0x000012d6                ks0108SelectFont
                0x00001202                ks0108SetDot
                0x0000197a                ks0108Enable
                0x00001634                ks0108Puts_P
                0x00000748                ks0108DrawLine
 .text          0x00001d72      0x51c touch.o
                0x00001ef4                F_radek
                0x00002042                F_stlaceno
                0x00001d72                Touch_init
 .text          0x0000228e        0x0 e:/winavr-20071221/bin/../lib/gcc/avr/4.2.2/avr5\libgcc.a(_divmodhi4.o)
 .text          0x0000228e        0x0 e:/winavr-20071221/bin/../lib/gcc/avr/4.2.2/avr5\libgcc.a(_exit.o)
 .text          0x0000228e        0x0 e:/winavr-20071221/bin/../lib/gcc/avr/4.2.2/avr5\libgcc.a(_copy_data.o)
 .text          0x0000228e        0x0 e:/winavr-20071221/bin/../lib/gcc/avr/4.2.2/avr5\libgcc.a(_clear_bss.o)
 .text          0x0000228e       0x4c e:/winavr-20071221/bin/../lib/gcc/avr/4.2.2/avr5\libgcc.a(_fixunssfsi.o)
                0x0000228e                __fixunssfsi
 .text          0x000022da      0x348 e:/winavr-20071221/bin/../lib/gcc/avr/4.2.2/avr5\libgcc.a(_addsub_sf.o)
                0x00002566                __subsf3
                0x000025c8                __addsf3
 .text          0x00002622      0x1fe e:/winavr-20071221/bin/../lib/gcc/avr/4.2.2/avr5\libgcc.a(_mul_sf.o)
                0x00002622                __mulsf3
 .text          0x00002820       0x6c e:/winavr-20071221/bin/../lib/gcc/avr/4.2.2/avr5\libgcc.a(_gt_sf.o)
                0x00002820                __gtsf2
 .text          0x0000288c       0x6c e:/winavr-20071221/bin/../lib/gcc/avr/4.2.2/avr5\libgcc.a(_ge_sf.o)
                0x0000288c                __gesf2
 .text          0x000028f8       0x6c e:/winavr-20071221/bin/../lib/gcc/avr/4.2.2/avr5\libgcc.a(_lt_sf.o)
                0x000028f8                __ltsf2
 .text          0x00002964       0xa6 e:/winavr-20071221/bin/../lib/gcc/avr/4.2.2/avr5\libgcc.a(_sf_to_si.o)
                0x00002964                __fixsfsi
 .text          0x00002a0a        0x0 e:/winavr-20071221/bin/../lib/gcc/avr/4.2.2/avr5\libgcc.a(_thenan_sf.o)
 .text          0x00002a0a        0x0 e:/winavr-20071221/bin/../lib/gcc/avr/4.2.2/avr5\libgcc.a(_udivmodhi4.o)
 .text          0x00002a0a        0x0 e:/winavr-20071221/bin/../lib/gcc/avr/4.2.2/avr5\libgcc.a(_prologue.o)
 .text          0x00002a0a        0x0 e:/winavr-20071221/bin/../lib/gcc/avr/4.2.2/avr5\libgcc.a(_epilogue.o)
 .text          0x00002a0a      0x1c0 e:/winavr-20071221/bin/../lib/gcc/avr/4.2.2/avr5\libgcc.a(_pack_sf.o)
                0x00002a0a                __pack_f
 .text          0x00002bca       0xe0 e:/winavr-20071221/bin/../lib/gcc/avr/4.2.2/avr5\libgcc.a(_unpack_sf.o)
                0x00002bca                __unpack_f
 .text          0x00002caa       0xac e:/winavr-20071221/bin/../lib/gcc/avr/4.2.2/avr5\libgcc.a(_fpcmp_parts_sf.o)
                0x00002caa                __fpcmp_parts_f
 .text          0x00002d56       0x42 e:/winavr-20071221/bin/../lib/gcc/avr/4.2.2/../../../../avr/lib/avr5\libc.a(itoa.o)
                0x00002d56                itoa
 .text          0x00002d98       0x20 e:/winavr-20071221/bin/../lib/gcc/avr/4.2.2/../../../../avr/lib/avr5\libc.a(strrev.o)
                0x00002d98                strrev
                0x00002db8                . = ALIGN (0x2)
 *(.text.*)
 .text.libgcc   0x00002db8       0x26 e:/winavr-20071221/bin/../lib/gcc/avr/4.2.2/avr5\libgcc.a(_divmodhi4.o)
                0x00002db8                __divmodhi4
                0x00002db8                _div
 .text.libgcc   0x00002dde        0x0 e:/winavr-20071221/bin/../lib/gcc/avr/4.2.2/avr5\libgcc.a(_exit.o)
 .text.libgcc   0x00002dde        0x0 e:/winavr-20071221/bin/../lib/gcc/avr/4.2.2/avr5\libgcc.a(_copy_data.o)
 .text.libgcc   0x00002dde        0x0 e:/winavr-20071221/bin/../lib/gcc/avr/4.2.2/avr5\libgcc.a(_clear_bss.o)
 .text.libgcc   0x00002dde       0x28 e:/winavr-20071221/bin/../lib/gcc/avr/4.2.2/avr5\libgcc.a(_udivmodhi4.o)
                0x00002dde                __udivmodhi4
 .text.libgcc   0x00002e06       0x38 e:/winavr-20071221/bin/../lib/gcc/avr/4.2.2/avr5\libgcc.a(_prologue.o)
                0x00002e06                __prologue_saves__
 .text.libgcc   0x00002e3e       0x36 e:/winavr-20071221/bin/../lib/gcc/avr/4.2.2/avr5\libgcc.a(_epilogue.o)
                0x00002e3e                __epilogue_restores__
                0x00002e74                . = ALIGN (0x2)
 *(.fini9)
 .fini9         0x00002e74        0x0 e:/winavr-20071221/bin/../lib/gcc/avr/4.2.2/avr5\libgcc.a(_exit.o)
                0x00002e74                exit
                0x00002e74                _exit
 *(.fini9)
 *(.fini8)
 *(.fini8)
 *(.fini7)
 *(.fini7)
 *(.fini6)
 *(.fini6)
 *(.fini5)
 *(.fini5)
 *(.fini4)
 *(.fini4)
 *(.fini3)
 *(.fini3)
 *(.fini2)
 *(.fini2)
 *(.fini1)
 *(.fini1)
 *(.fini0)
 .fini0         0x00002e74        0x2 e:/winavr-20071221/bin/../lib/gcc/avr/4.2.2/avr5\libgcc.a(_exit.o)
 *(.fini0)
                0x00002e76                _etext = .

.data           0x00800060        0x8 load address 0x00002e76
                0x00800060                PROVIDE (__data_start, .)
 *(.data)
 .data          0x00800060        0x0 e:/winavr-20071221/bin/../lib/gcc/avr/4.2.2/../../../../avr/lib/avr5/crtm16.o
 .data          0x00800060        0x0 komparator.o
 .data          0x00800060        0x0 ks0108.o
 .data          0x00800060        0x0 touch.o
 .data          0x00800060        0x0 e:/winavr-20071221/bin/../lib/gcc/avr/4.2.2/avr5\libgcc.a(_divmodhi4.o)
 .data          0x00800060        0x0 e:/winavr-20071221/bin/../lib/gcc/avr/4.2.2/avr5\libgcc.a(_exit.o)
 .data          0x00800060        0x0 e:/winavr-20071221/bin/../lib/gcc/avr/4.2.2/avr5\libgcc.a(_copy_data.o)
 .data          0x00800060        0x0 e:/winavr-20071221/bin/../lib/gcc/avr/4.2.2/avr5\libgcc.a(_clear_bss.o)
 .data          0x00800060        0x0 e:/winavr-20071221/bin/../lib/gcc/avr/4.2.2/avr5\libgcc.a(_fixunssfsi.o)
 .data          0x00800060        0x0 e:/winavr-20071221/bin/../lib/gcc/avr/4.2.2/avr5\libgcc.a(_addsub_sf.o)
 .data          0x00800060        0x0 e:/winavr-20071221/bin/../lib/gcc/avr/4.2.2/avr5\libgcc.a(_mul_sf.o)
 .data          0x00800060        0x0 e:/winavr-20071221/bin/../lib/gcc/avr/4.2.2/avr5\libgcc.a(_gt_sf.o)
 .data          0x00800060        0x0 e:/winavr-20071221/bin/../lib/gcc/avr/4.2.2/avr5\libgcc.a(_ge_sf.o)
 .data          0x00800060        0x0 e:/winavr-20071221/bin/../lib/gcc/avr/4.2.2/avr5\libgcc.a(_lt_sf.o)
 .data          0x00800060        0x0 e:/winavr-20071221/bin/../lib/gcc/avr/4.2.2/avr5\libgcc.a(_sf_to_si.o)
 .data          0x00800060        0x8 e:/winavr-20071221/bin/../lib/gcc/avr/4.2.2/avr5\libgcc.a(_thenan_sf.o)
                0x00800060                __thenan_sf
 .data          0x00800068        0x0 e:/winavr-20071221/bin/../lib/gcc/avr/4.2.2/avr5\libgcc.a(_udivmodhi4.o)
 .data          0x00800068        0x0 e:/winavr-20071221/bin/../lib/gcc/avr/4.2.2/avr5\libgcc.a(_prologue.o)
 .data          0x00800068        0x0 e:/winavr-20071221/bin/../lib/gcc/avr/4.2.2/avr5\libgcc.a(_epilogue.o)
 .data          0x00800068        0x0 e:/winavr-20071221/bin/../lib/gcc/avr/4.2.2/avr5\libgcc.a(_pack_sf.o)
 .data          0x00800068        0x0 e:/winavr-20071221/bin/../lib/gcc/avr/4.2.2/avr5\libgcc.a(_unpack_sf.o)
 .data          0x00800068        0x0 e:/winavr-20071221/bin/../lib/gcc/avr/4.2.2/avr5\libgcc.a(_fpcmp_parts_sf.o)
 .data          0x00800068        0x0 e:/winavr-20071221/bin/../lib/gcc/avr/4.2.2/../../../../avr/lib/avr5\libc.a(itoa.o)
 .data          0x00800068        0x0 e:/winavr-20071221/bin/../lib/gcc/avr/4.2.2/../../../../avr/lib/avr5\libc.a(strrev.o)
 *(.data*)
 *(.rodata)
 *(.rodata*)
 *(.gnu.linkonce.d*)
                0x00800068                . = ALIGN (0x2)
                0x00800068                _edata = .
                0x00800068                PROVIDE (__data_end, .)

.bss            0x00800068        0xb load address 0x00002e7e
                0x00800068                PROVIDE (__bss_start, .)
 *(.bss)
 .bss           0x00800068        0x0 e:/winavr-20071221/bin/../lib/gcc/avr/4.2.2/../../../../avr/lib/avr5/crtm16.o
 .bss           0x00800068        0x2 komparator.o
                0x00800069                j
                0x00800068                preruseni
 .bss           0x0080006a        0x1 ks0108.o
                0x0080006a                ks0108Inverted
 .bss           0x0080006b        0x0 touch.o
 .bss           0x0080006b        0x0 e:/winavr-20071221/bin/../lib/gcc/avr/4.2.2/avr5\libgcc.a(_divmodhi4.o)
 .bss           0x0080006b        0x0 e:/winavr-20071221/bin/../lib/gcc/avr/4.2.2/avr5\libgcc.a(_exit.o)
 .bss           0x0080006b        0x0 e:/winavr-20071221/bin/../lib/gcc/avr/4.2.2/avr5\libgcc.a(_copy_data.o)
 .bss           0x0080006b        0x0 e:/winavr-20071221/bin/../lib/gcc/avr/4.2.2/avr5\libgcc.a(_clear_bss.o)
 .bss           0x0080006b        0x0 e:/winavr-20071221/bin/../lib/gcc/avr/4.2.2/avr5\libgcc.a(_fixunssfsi.o)
 .bss           0x0080006b        0x0 e:/winavr-20071221/bin/../lib/gcc/avr/4.2.2/avr5\libgcc.a(_addsub_sf.o)
 .bss           0x0080006b        0x0 e:/winavr-20071221/bin/../lib/gcc/avr/4.2.2/avr5\libgcc.a(_mul_sf.o)
 .bss           0x0080006b        0x0 e:/winavr-20071221/bin/../lib/gcc/avr/4.2.2/avr5\libgcc.a(_gt_sf.o)
 .bss           0x0080006b        0x0 e:/winavr-20071221/bin/../lib/gcc/avr/4.2.2/avr5\libgcc.a(_ge_sf.o)
 .bss           0x0080006b        0x0 e:/winavr-20071221/bin/../lib/gcc/avr/4.2.2/avr5\libgcc.a(_lt_sf.o)
 .bss           0x0080006b        0x0 e:/winavr-20071221/bin/../lib/gcc/avr/4.2.2/avr5\libgcc.a(_sf_to_si.o)
 .bss           0x0080006b        0x0 e:/winavr-20071221/bin/../lib/gcc/avr/4.2.2/avr5\libgcc.a(_thenan_sf.o)
 .bss           0x0080006b        0x0 e:/winavr-20071221/bin/../lib/gcc/avr/4.2.2/avr5\libgcc.a(_udivmodhi4.o)
 .bss           0x0080006b        0x0 e:/winavr-20071221/bin/../lib/gcc/avr/4.2.2/avr5\libgcc.a(_prologue.o)
 .bss           0x0080006b        0x0 e:/winavr-20071221/bin/../lib/gcc/avr/4.2.2/avr5\libgcc.a(_epilogue.o)
 .bss           0x0080006b        0x0 e:/winavr-20071221/bin/../lib/gcc/avr/4.2.2/avr5\libgcc.a(_pack_sf.o)
 .bss           0x0080006b        0x0 e:/winavr-20071221/bin/../lib/gcc/avr/4.2.2/avr5\libgcc.a(_unpack_sf.o)
 .bss           0x0080006b        0x0 e:/winavr-20071221/bin/../lib/gcc/avr/4.2.2/avr5\libgcc.a(_fpcmp_parts_sf.o)
 .bss           0x0080006b        0x0 e:/winavr-20071221/bin/../lib/gcc/avr/4.2.2/../../../../avr/lib/avr5\libc.a(itoa.o)
 .bss           0x0080006b        0x0 e:/winavr-20071221/bin/../lib/gcc/avr/4.2.2/../../../../avr/lib/avr5\libc.a(strrev.o)
 *(.bss*)
 *(COMMON)
 COMMON         0x0080006b        0x8 ks0108.o
                0x0080006b                ks0108FontColor
                0x0080006c                ks0108Coord
                0x0080006f                ks0108FontRead
                0x00800071                ks0108Font
                0x00800073                PROVIDE (__bss_end, .)
                0x00002e76                __data_load_start = LOADADDR (.data)
                0x00002e7e                __data_load_end = (__data_load_start + SIZEOF (.data))

.noinit         0x00800073        0x0
                0x00800073                PROVIDE (__noinit_start, .)
 *(.noinit*)
                0x00800073                PROVIDE (__noinit_end, .)
                0x00800073                _end = .
                0x00800073                PROVIDE (__heap_start, .)

.eeprom         0x00810000        0x0
 *(.eeprom*)
                0x00810000                __eeprom_end = .

.fuse
 *(.fuse)
 *(.lfuse)
 *(.hfuse)
 *(.efuse)

.lock
 *(.lock*)

.signature
 *(.signature*)

.stab           0x00000000      0x378
 *(.stab)
 .stab          0x00000000      0x378 e:/winavr-20071221/bin/../lib/gcc/avr/4.2.2/../../../../avr/lib/avr5/crtm16.o

.stabstr        0x00000000       0x5f
 *(.stabstr)
 .stabstr       0x00000000       0x5f e:/winavr-20071221/bin/../lib/gcc/avr/4.2.2/../../../../avr/lib/avr5/crtm16.o

.stab.excl
 *(.stab.excl)

.stab.exclstr
 *(.stab.exclstr)

.stab.index
 *(.stab.index)

.stab.indexstr
 *(.stab.indexstr)

.comment
 *(.comment)

.debug
 *(.debug)

.line
 *(.line)

.debug_srcinfo
 *(.debug_srcinfo)

.debug_sfnames
 *(.debug_sfnames)

.debug_aranges  0x00000000       0x60
 *(.debug_aranges)
 .debug_aranges
                0x00000000       0x20 komparator.o
 .debug_aranges
                0x00000020       0x20 ks0108.o
 .debug_aranges
                0x00000040       0x20 touch.o

.debug_pubnames
                0x00000000      0x2a6
 *(.debug_pubnames)
 .debug_pubnames
                0x00000000       0x4e komparator.o
 .debug_pubnames
                0x0000004e      0x21c ks0108.o
 .debug_pubnames
                0x0000026a       0x3c touch.o

.debug_info     0x00000000     0x118f
 *(.debug_info)
 .debug_info    0x00000000      0x22e komparator.o
 .debug_info    0x0000022e      0xc66 ks0108.o
 .debug_info    0x00000e94      0x2fb touch.o
 *(.gnu.linkonce.wi.*)

.debug_abbrev   0x00000000      0x2f7
 *(.debug_abbrev)
 .debug_abbrev  0x00000000       0xb5 komparator.o
 .debug_abbrev  0x000000b5      0x175 ks0108.o
 .debug_abbrev  0x0000022a       0xcd touch.o

.debug_line     0x00000000     0x11b3
 *(.debug_line)
 .debug_line    0x00000000      0x1b1 komparator.o
 .debug_line    0x000001b1      0xc34 ks0108.o
 .debug_line    0x00000de5      0x3ce touch.o

.debug_frame    0x00000000      0x1f0
 *(.debug_frame)
 .debug_frame   0x00000000       0x40 komparator.o
 .debug_frame   0x00000040      0x170 ks0108.o
 .debug_frame   0x000001b0       0x40 touch.o

.debug_str      0x00000000       0x49
 *(.debug_str)
 .debug_str     0x00000000       0x49 ks0108.o

.debug_loc
 *(.debug_loc)

.debug_macinfo
 *(.debug_macinfo)
OUTPUT(komparator.elf elf32-avr)
LOAD linker stubs
